:1000000018308A000E2E0000FF00030E8301A100AD
:100010000A08A0008A010408A2007708A300780853
:10002000A4007908A5007A08A6007B08A70083131E
:1000300083128C308400801E1F288C1A32282208DC
:1000400084002308F7002408F8002508F900260892
:10005000FA002708FB0020088A00210E8300FF0E0B
:100060007F0E09008A110A12EF280A108A100A115D
:1000700082074F344E3434344934593420345234A6
:1000800042344F3458342D343334313420344434F2
:10009000573400340A108A100A1182074E344F3444
:1000A0002034573441345234523441344E34543471
:1000B00049344534533420344F34523400340A1018
:1000C0008A100A118207203443344F344D344D34A2
:1000D000453452344334493441344C34203455345B
:1000E00053344534203400340A108A100A11820730
:1000F00020344F34203400340A108A100A11820749
:1001000020344534203400340A108A100A11820742
:100110002034203400340A108A100A118207203457
:10012000533441345434533400340A108A100A11C1
:100130008207483444344F345034203400340A1099
:100140008A100A11820753344534523449344134F9
:100150004C3420344F344B3400340A108A100A11C6
:1001600082074E344F3454342034413420344734E1
:100170005034533400340A108A100A11820747346D
:1001800050345334203446344F3455344E34443490
:1001900000340A108A100A1182074734503452344E
:1001A0004D34433420345034463400340A108A101D
:1001B0000A118207473450344734473441342034DD
:1001C0005034463400340A108A100A1182074E3423
:1001D0004F3420344734503453343F340034831682
:1001E00086108312861428302C0784008C1EF62873
:1001F0001A0880002C088316E900013083122C07AE
:100200000339AC002D082C02031D0A298316690846
:100210008312AC0083168610831286108C128A110A
:100220000A121F28643084000008031926290130AF
:10023000F800F701F70B1A29F80B19294A30F700D3
:10024000F70B202900000000800B172900340D3027
:10025000F700F70B292974081039003A031D3229D9
:100260000812332908168316081274082039003A38
:10027000031D3E2983128812402983168312881693
:100280008316881274084039003A031D4B298312E3
:1002900008134D2983168312081783160813740850
:1002A0008039003A031D5829831288135A2983166E
:1002B0008312881783168813881183128815831672
:1002C00088118312881174080139003A031D6A29C4
:1002D00008126B2908168316081274080239003AAE
:1002E000031D7629831288127829831683128816B3
:1002F0008316881274080439003A031D8329831277
:1003000008138529831683120817831608137408A7
:100310000839003A031D9029831288139229831605
:100320008312881783168813881183128815831601
:100330008811831288110034831688108312881064
:100340000830F40027210130F40027210230E400B6
:1003500012210230F40027210230E400122106307D
:10036000F40027210C30F40027210230E400122190
:10037000003483168810831288147308F400272130
:100380000034831688108312881080306B07EC00CD
:10039000F4002721003483161F149F141F159F118A
:1003A00083121F108316091283129412DD125D0846
:1003B0008316870083125D165D08831687008312FB
:1003C000DD115D08831687000030831294008316C8
:1003D00094000108C7390838810083129001003069
:1003E000F800920000308316920083125D155D08BC
:1003F00083168700831297019701DD145D08831629
:10040000870083129D019D01073083169C0005081B
:100410000330F700F70B0A2A1C0883120D1383160A
:100420009D018C16C03083128B0483160610831234
:100430000614831686108312861083160611831203
:1004400006118316861183128611831606128312F3
:10045000061283168612831286120330E300831677
:1004600088108312881083168811831288118316CE
:100470000811831208110F30E400122163080139BA
:10048000003A031D452A0812462A08168316081248
:10049000831263080239003A031D502A8812512A38
:1004A000881683168812831263080439003A031DE4
:1004B0005B2A08135C2A0817831608138312630843
:1004C0000839003A031D662A8813672A881783169D
:1004D0008813881183128815831688118312881156
:1004E0000530E400122163080139003A031D7A2A1D
:1004F00008127B2A08168316081283126308023931
:10050000003A031D852A8812862A881683168812C7
:10051000831263080439003A031D902A0813912AB4
:10052000081783160813831263080839003A031D5D
:100530009B2A88139C2A8817831688138811831294
:10054000881583168811831288110530E400122162
:1005500063080139003A031DAF2A0812B02A0816B1
:1005600083160812831263080239003A031DBA2A5F
:100570008812BB2A881683168812831263080439EE
:10058000003A031DC52A0813C62A08178316081344
:10059000831263080839003A031DD02A8813D12A30
:1005A000881783168813881183128815831688117B
:1005B000831288110530E4001221081283160812F4
:1005C0008312881683168812831208138316081361
:1005D0008312881383168813881183128815831653
:1005E0008811831288112830F40027219C21E3010F
:1005F0006308352000380319012BE30AF300B92101
:10060000F82A0330E300FA30E4001221E30B032B55
:100610004030EB00C121E30163084A200038031990
:10062000152BE30AF300B9210C2B83160610831255
:1006300006100230E300FA30E4001221E30B1B2B1A
:1006400083160610831206104030EB00C121E3012F
:1006500063085F2000380319312BE30AF300B92146
:10066000282B0230E300FA30E4001221E30B332B95
:1006700083160610831206148A150A16312E2D08C9
:100680002C0203193F2B28302D0784000008EB00B3
:1006900001302D070339AD006B08F80000346910F4
:1006A000E801E8016808E80A003A0319642B63309E
:1006B0006807EA003F236A08840078088000680819
:1006C000033C031C0030522B6918872B3F2378080A
:1006D000E7006308473C031D7D2B6408503C031D65
:1006E0007D2B6508523C031D7D2B66084D3C031D88
:1006F0007D2B6708433C03196914E80A6408E3008A
:100700006508E4006608E5006708E600642B003031
:1007100069180130F80000343F237808E4006408C9
:100720002C3C0319972B3F237808E4008F2B0034CF
:100730003F233F237808AE003F237808AF003F23D4
:100740007808B0003F237808B1003F237808B20052
:100750003F237808B3000230B30730303302093C3E
:100760000318B52B0A30B302B20A30303202053C0E
:100770000318BD2B3030B200B10A30303102093CD1
:100780000318C52B0A30B102B00A30303002053CE4
:100790000318CD2B3030B000AF0A8C233F237808EC
:1007A000413C031DD52B5C14D62B5C108C233F23BE
:1007B0007808B4003F237808B5003F237808B600D6
:1007C0003F237808B7003F233F237808B8008C23E5
:1007D0008C233F237808B9003F237808BA003F23D1
:1007E0007808BB003F237808BC003F237808BD0091
:1007F0008C233F237808BE008C238C238C233F233B
:100800007808BF003F237808C0003F237808C10064
:100810003F237808C2008A150A16E12EF701F80175
:10082000700803107118F707F70CF80CF118F707A8
:10083000F70CF80C7119F707F70CF80CF119F7071A
:10084000F70CF80C711AF707F70CF80CF11AF70708
:10085000F70CF80C711BF707F70CF80CF11BF707F6
:10086000F70CF80C00348E30F70083165308F800AC
:100870005208F900FA01F808031D482C7908F8001D
:10088000F9010830F702F808031D482CF701502C35
:100890000310F81B4F2CF90DF80DF703482CF81333
:1008A0000000831200348030831C592C8316D80634
:1008B00083128316DD01DE015408DC005808DC06D3
:1008C00053080319442DDB00F700570803194D2D79
:1008D000DB020319EA2C031CA92C5808E100E117DC
:1008E0005908E0005A08DF00DE010310E10CE00CBB
:1008F000DF0CDE0CDB0B742CDC1F812C5D14612DF6
:100900005D105B105D16D6308400762D5D12DC1B09
:10091000932C5B1C9E2CE10CE00CDF0CDE0CF70A28
:1009200003195C2D9E2CE11BA12C0310DE0DDF0DA5
:10093000E00DE10DF70303195C2D932C5D17092DD4
:100940005D135408DC00D41FA72CE117552DE113CB
:10095000552D5708DB00F7005308DB025408E1006F
:10096000E1175508E0005608DF00DE010310E10C36
:10097000E00CDF0CDE0CDB0BB52CDC1FC22CDD1415
:10098000612DDD105B10DD16DA308400762DDD126E
:10099000DC1BD42C5B1CDF2CE10CE00CDF0CDE0C30
:1009A000F70A03195C2DDF2CE11BE22C0310DE0D8E
:1009B000DF0DE00DE10DF70303195C2DD42CDD17DD
:1009C000092DDD135808DC00D81FE82CE117552D40
:1009D000E113552D5808E100E1175908E0005A08C5
:1009E000DF00DC1FF72CE1135D15612D5D11DE01C9
:1009F0005B10D6308400762DDC1B1F2D5408DC00E4
:100A00005B1C092DE10CE00CDF0CDE0CF70A03196E
:100A10005C2DDE1F1A2DDF0A031D1A2DE00A031DAF
:100A20001A2DE10A031D1A2DE10CE00CDF0CF70A68
:100A300003195C2D5D1BA02CDD1BE12C3E2D8030AD
:100A4000E106E11F272D612D5808DC00342D5408E4
:100A5000DC00E108031D342DE008031D342DDF0800
:100A6000031D342DF701552DE11B3E2D0310DE0D26
:100A7000DF0DE00DE10DF70B342D5C2DDC1F422D59
:100A8000E117552DE113552D5708F7005808E100DF
:100A90005908E0005A08DF00552D5308F7005408A4
:100AA000E1005508E0005608DF006108F800600822
:100AB000F9005F08FA00942DF701F801F901FA0135
:100AC000942DDE01DF09E009E109DE09DE0A031DDC
:100AD0006F2DDF0A031D6F2DE00A0319E10A5D186F
:100AE000802CDD18C12C5D19F62C242D0008DF07A1
:100AF000031C802DE00A031D802DE10A03195B14FD
:100B000084030008E007031C882DE10A03195B1425
:100B100084030008801F803AE10703185B145D1A04
:100B2000862CDD1AC72CFC2C00008312003483169F
:100B30004E0803195D2EDA00520803195D2EDA0201
:100B4000031CA72D7F30DA0703185D2EAD2D8130F1
:100B5000DA02031C5D2E03195D2E5A08F700F80116
:100B6000F901FA01D9014F08D800D8175008D70069
:100B70005108D6001930DA005508D6020318D02DD6
:100B80000130D7020318D02DD8020318D02DD90276
:100B90000318D02DD90AD80AD70A5508D607022E2D
:100BA0005408D7020318EB2D0130D8020318EB2D9F
:100BB000D9020318EB2DD90AD80A5408D7075508CB
:100BC000D607031C022ED70A031D022ED80A031DC6
:100BD000022ED90A022E53088038D8020318012E9B
:100BE0000130D9020318012ED90A53088038D807DA
:100BF0005408D707031CDF2DD80A031DDF2DD90A9F
:100C0000DF2D7A14DA0B052E102E0310D60DD70D1A
:100C1000D80DD90D0310FA0DF90DF80DDB0DBC2D13
:100C20005B1C182E0310F80CF90CFA0CDB0C1B2EB5
:100C3000F70303195D2EDB1B442E0310D60DD70DD1
:100C4000D80DD90D5508D6020318302E0130D70221
:100C50000318302ED8020318302ED902031C532E4D
:100C60005408D70203183B2E0130D80203183B2E3C
:100C7000D902031C532E53088038D8020318442E7F
:100C80000130D902031C532EFA0A031D532EF90A10
:100C9000031D532EF80A031D532EF70A03195D2E68
:100CA000F80CF90CFA0C4F08DA005308DA06DA1FD0
:100CB0005B2EF817612EF813612EF701F801F90188
:100CC000FA01000083120034831652080319D52E4E
:100CD000DA0056080319D52EDA070318762E7F306E
:100CE000DA02031CD52E0319D52E7A2E8130DA07AD
:100CF0000318D52E5A08F700F801F901FA01530834
:100D0000DE00DE175408DD005508DC001830DA007C
:100D1000DB015C1CA32E5908FA07031C952EF90A67
:100D2000031D952EF80A0319DB175808F907031C51
:100D30009C2EF80A0319DB175708D400D41754085F
:100D4000F8070318DB17DB0DF80CF90CFA0CDE0CB6
:100D5000DD0CDC0C0310DA0B882E0130F7070318CA
:100D6000D52EF81BBA2EDE0DFA0DF90DF80DF7038E
:100D70000319D52EDE1FCB2EFA0A031DCB2EF90A3E
:100D8000031DCB2EF80A031DCB2EF80CF90CFA0C20
:100D9000F70A0319D52E5308DB005708DB06DB1FC3
:100DA000D32EF817D92EF813D92EF701F801F9012F
:100DB000FA0100008312003483164F08D60053084E
:100DC000D606D61FE82E03110310CF1B03141B2FCA
:100DD0004F08D6005208D7004E08D7020319F62E46
:100DE000D61F1B2F0308013A83001B2F5308D7007F
:100DF0004F08D7020319022FD61F1B2F0308013AF1
:100E000083001B2F5408D7005008D70203190E2F58
:100E1000D61F1B2F0308013A83001B2F5508D7004C
:100E20005108D70203191A2FD61F1B2F0308013AA6
:100E300083001B2F0310831200348E30F7008316BB
:100E40004E08F7024F08F9005008F800F917F708A4
:100E50000319352F0310F908031D312FF808031962
:100E6000352FF90CF80CF70B2A2FCF1F3C2FF80960
:100E7000F909F80A0319F90A0000831200348314EF
:100E800083162308D6002208D5002108D4002008A4
:100E9000D300DB30DA000F30D9004930D8007F3082
:100EA000D7008312532477088316A4007808A5007E
:100EB0007908A6007A08A700AB002608AA00250832
:100EC000A9002408A8008A15831255218A1100342C
:100ED0007208F80171020318702F7108F7007C2F57
:100EE000F7010830F300F10DF70D720877020318CF
:100EF000F700F80DF30B732F00341030F700FA01F0
:100F0000EF01EC0CEB0C031C8B2F6D08FA07031898
:100F1000EF0A6E08EF07EF0CFA0CF90CF80CF70B60
:100F2000812F8A110A16FD28F801F901F701FA014B
:100F30006C08031D9E2F6B080319B82F1030ED00AD
:100F40000310E90DEA0DF70DFA0D6C087A02031D86
:100F5000AB2F6B087702031CB42F6B08F702031C3E
:100F6000FA036C08FA020314F80DF90DED0BA02F2B
:080F700000008A110A16E429B1
:1010000030304102E800F0000A30F1008A110E246D
:101010008A157808E900303042026907E300303071
:101020003F02E800F0000A30F1008A110E248A1510
:101030007808E900303040026907E4006308013AAB
:1010400003194428033A03194828013A03194D2883
:10105000073A03195228013A03195728033A03198A
:101060005C28013A031961280F3A03196628013AEE
:1010700003196B28033A03197028013A03197828D9
:10108000073A031980288828E6016408E5008B28C0
:101090001F306407E500E6018B283B306407E5005C
:1010A000E6018B285A306407E500E6018B2878308A
:1010B0006407E500E6018B2897306407E500E60148
:1010C0008B28B5306407E500E6018B28D43064072F
:1010D000E500E6018B28F3306407E500E6018B2884
:1010E00011306407E5000130E6000318E60A8B289A
:1010F00030306407E5000130E6000318E60A8B286B
:101100004E306407E5000130E6000318E60A8B283C
:10111000E6010130E50030302E02E800F0000A3030
:10112000F1008A110E248A157808E90030302F0268
:1011300069078316D301D2008A11831233248A15DA
:101140007A08D1007908D0007808CF007708CE005F
:1011500001306502E7006608E8000030031C01303A
:10116000E802831451088316D600831250088316B0
:10117000D50083124F088316D40083124E088316BD
:10118000D300DA01D9014030D8008230D7008A116B
:10119000831253248A157708E9007808EA00790851
:1011A000EB007A08EC008316D10083126B088316DB
:1011B000D00083126A088316CF0083126908831651
:1011C000CE00D501D4014030D3008330D2008A1143
:1011D000831297258A157708ED007808EE007908C4
:1011E000EF007A08F00068088316D30083126708BE
:1011F0008316D2008A11831233248A1583107A0849
:101200008316D6007908D5007808D4007708D30073
:101210007008DA0083126F088316D90083126E08F3
:101220008316D80083126D088316D7008A118312A3
:1012300053248A157708F1007808F2007908F30042
:101240007A08F4008316D1007308D0007208CF002A
:101250007108CE00D5018030D4003630D3008730FD
:10126000D2008A11831297258A15DB308316D500A8
:101270000F30D4004930D3008130D2007A08D90031
:101280007908D8007808D7007708D6008A11831229
:1012900064268A157A08D1007908D0007808CF0032
:1012A0007708CE008A150A16FA2E7F308316B4000E
:1012B000B501B601B7017E30BE008030BF00C0016D
:1012C000C1017A30C2002A30C300AA30C400A33062
:1012D000C5007530C600B630C7000930C8009C3064
:1012E000C9006F30CA004F30CB00B430CC000B3097
:1012F000CD002B08D1002A08D0002908CF002808EB
:10130000CE00D501D401D301D2018A118312DC268B
:101310008A15031C8F2980308316A9068312831631
:101320002B08D1002A08D0002908CF002808CE00B9
:10133000DB30D5000F30D4004930D3007F30D200ED
:101340008A11831297258A157A088316D1007908A5
:10135000D0007808CF007708CE008A1183121D27AD
:101360008A1578088316B8002B08D1002A08D00007
:101370002908CF002808CE00DB30D5000F30D4007C
:101380004930D3007F30D2008A11831297258A1505
:1013900077088316CE007808CF007908D0007A0845
:1013A000D100D3013808D2008A11831233248A1560
:1013B000831483165108D6005008D5004F08D40076
:1013C0004E08D3007A08DA007908D9007808D800E6
:1013D0007708D7008A11831253248A157A08831656
:1013E000BD007908BC007808BB007708BA0003305C
:1013F000B805B8080319002A3808023C031D1E2A44
:101400003D08D5003C08D4003B08D3003A08D20080
:10141000DB30D9000F30D8004930D7007F30D600FC
:101420008A11831264268A157A088316B300790814
:10143000B2007808B1007708B0008F2A380B582A1C
:101440008314D601D501D4017F30D3003D08DA00E2
:101450003C08D9003B08D8003A08D7008A1183120B
:1014600053248A1577088316CE007808CF007908B0
:10147000D0007A08D100D5005008D4004F08D3001E
:101480004E08D200DB30D9000F30D8004930D700E9
:101490007F30D6008A11831264268A157A08831653
:1014A000B3007908B2007808B1007708B0008F2A3D
:1014B00083143D08D6003C08D5003B08D4003A0808
:1014C000D300DA01D901D8017F30D7008A11831205
:1014D00053248A1577088316CE007808CF00790840
:1014E000D0007A08D100D5005008D4004F08D300AE
:1014F0004E08D200DB30D9000F30D8004930D70079
:101500007F30D6008A11831264268A157A088316E2
:10151000B3007908B2007808B1007708B000AF01D5
:10152000AE01AD017F30AC003308D5003208D400E5
:101530003108D3003008D2003308D9003208D8006F
:101540003108D7003008D6008A11831264268A1524
:101550007A088316B3007908B2007808B1007708DA
:10156000B000B9013908033C031C1E2B3708D50015
:101570003608D4003508D3003408D2003308D90027
:101580003208D8003108D7003008D6008A118312FB
:1015900064268A157A088316B7007908B600780899
:1015A000B5007708B400390DF700F70DFC30F705EA
:1015B0007708BE3E84000008CE00840A0008CF00F1
:1015C000840A0008D000840A0008D100D500500821
:1015D000D4004F08D3004E08D2003708D90036088F
:1015E000D8003508D7003408D6008A118312642643
:1015F0008A1504088316D20083102F08D6002E08FF
:10160000D5002D08D4002C08D3007A08DA00790818
:10161000D9007808D8007708D7008A11831253249C
:101620008A158316520884007A08AF007908AE0044
:101630007808AD007708AC00B90AB22A3808023C35
:101640000319242B380B262B8030AD062C08F7000D
:101650002D08F8002E08F9002F08FA008312003434
:1016600051088316AB00831250088316AA00831218
:101670004F088316A90083124E088316A800831210
:1016800055217A08E6007908E5007808E400770833
:10169000E30051088316A300831250088316A200AA
:1016A00083124F088316A10083124E088316A000F0
:1016B0008A1183123F278A157A08EA007908E9001F
:1016C0007808E8007708E70051088316D5008312F0
:1016D00050088316D40083124F088316D300831258
:1016E0004E088316D200D901D801D7018030D60028
:1016F0008A11831264268A157708F3007808F400AB
:101700007908F5007A08F6008316AB007508AA0080
:101710007408A9007308A800831255217A08EE0006
:101720007908ED007808EC007708EB005108831683
:10173000D500831250088316D40083124F088316F5
:10174000D30083124E088316D200D901D801D701E5
:101750008030D6008A11831264268A157708F30038
:101760007808F4007908F5007A08F6008316A300DB
:101770007508A2007408A1007308A0008A118312E2
:101780003F278A157A08F2007908F1007808F000FE
:101790007708EF005230D5004930D4001D30D30017
:1017A0007130D200AE308316D500D730D4007430FB
:1017B000D3007530D200831266088316D9008312D5
:1017C00065088316D800831264088316D700831235
:1017D00063088316D6008A11831264268A15831043
:1017E00055088316D600831254088316D500831239
:1017F00053088316D400831252088316D3007A0844
:10180000DA007908D9007808D8007708D7008A115B
:10181000831253248A157A08D5007908D4007808F1
:10182000D3007708D2002C308316D5006330D40063
:101830000330D3007A30D20083126A088316D900AD
:10184000831269088316D800831268088316D700AC
:10185000831267088316D6008A11831264268A15BC
:10186000831455088316D600831254088316D500B6
:10187000831253088316D400831252088316D300B0
:101880007A08DA007908D9007808D8007708D700F4
:101890008A11831253248A157A08D5007908D40056
:1018A0007808D3007708D200C1308316D500733092
:1018B000D4006F30D3007830D20083126E088316C4
:1018C000D90083126D088316D80083126C08831622
:1018D000D70083126B088316D6008A118312642600
:1018E0008A15831455088316D6008312540883166C
:1018F000D500831253088316D4008312520883162E
:10190000D3007A08DA007908D9007808D800770877
:10191000D7008A11831253248A157A08D5007908D2
:10192000D4007808D3007708D20048308316D50059
:101930005130D4002730D3007A30D2007208D90059
:101940007108D8007008D70083126F088316D6007C
:101950008A11831264268A15831455088316D600CB
:10196000831254088316D500831253088316D400BB
:10197000831252088316D3007A08DA007908D90056
:101980007808D8007708D7008A11831253248A1563
:101990007A08D5007908D4007808D3007708D200F7
:1019A00055088316D500831254088316D400831279
:1019B00053088316D300831252088316D2001430C2
:1019C000D9002E30D8006530D7008630D6008A1175
:1019D000831264268A157A08D5007908D40078081D
:1019E000D3007708D2008A150A16FD2E51088316F7
:1019F000AB00831250088316AA0083124F08831687
:101A0000A90083124E088316A800831255217A0874
:101A1000E6007908E5007808E4007708E30051085B
:101A20008316A300831250088316A20083124F0866
:101A30008316A10083124E088316A0008A11831218
:101A40003F278A157A08EA007908E9007808E80053
:101A50007708E70051088316D500831250088316D3
:101A6000D40083124F088316D30083124E088316C6
:101A7000D200D901D801D7018030D6008A11831253
:101A800064268A157708F3007808F4007908F500D1
:101A90007A08F6008316AB007908AA007808A90036
:101AA0007708A800831255217A08EE007908ED0026
:101AB0007808EC007708EB0051088316D5008312F4
:101AC00050088316D40083124F088316D300831264
:101AD0004E088316D200D901D801D7018030D60034
:101AE0008A11831264268A157708F3007808F400B7
:101AF0007908F5007A08F6008316A3007908A20099
:101B00007808A1007708A0008A1183123F278A1560
:101B10007A08F2007908F1007808F0007708EF0001
:101B20006430D900B030D8006230D7007730D600AA
:101B300044308316D500C130D4004C30D3007D3002
:101B4000D200831266088316D900831265088316B3
:101B5000D800831264088316D700831263088316A3
:101B6000D6008A11831264268A15831459088316B5
:101B7000D600831258088316D5008312570883169F
:101B8000D400831256088316D3007A08DA00790845
:101B9000D9007808D8007708D7008A118312532417
:101BA0008A157A08D9007908D8007808D70077080C
:101BB000D600E7308316D500E230D4000F30D300D2
:101BC0007B30D20083126A088316D9008312690819
:101BD0008316D800831268088316D700831267081B
:101BE0008316D6008A11831264268A158310590839
:101BF0008316D600831258088316D500831257081F
:101C00008316D400831256088316D3007A08DA00AC
:101C10007908D9007808D8007708D7008A1183128C
:101C200053248A157A08D9007908D8007808D70093
:101C30007708D60036308316D5007230D4005D3078
:101C4000D3007730D20083126E088316D900831236
:101C50006D088316D80083126C088316D700831290
:101C60006B088316D6008A11831264268A158314A2
:101C700059088316D600831258088316D50083129C
:101C800057088316D400831256088316D3007A08A7
:101C9000DA007908D9007808D8007708D7008A11C7
:101CA000831253248A157A08D9007908D800780855
:101CB000D7007708D600BD308316D500C330D400D6
:101CC0006D30D3007430D2007208D9007108D8008A
:101CD0007008D70083126F088316D6008A1183120A
:101CE00064268A15831059088316D6008312580873
:101CF0008316D500831257088316D4008312560822
:101D00008316D3007A08DA007908D9007808D80059
:101D10007708D7008A11831253248A157A08D900CC
:101D20007908D8007808D7007708D6008316D5013F
:101D3000D4014030D3008030D20083125108831682
:101D4000D900831250088316D80083124F088316D7
:101D5000D70083124E088316D6008A118312642698
:101D60008A157708F3007808F4007908F5007A08F6
:101D7000F6008316AB007908AA007808A900770856
:101D8000A8008312552127308316D500C030D40017
:101D90003030D3007630D2007A08D9007908D800E4
:101DA0007808D7007708D6008A11831264268A152E
:101DB0000408F400831459088316D60083125808C7
:101DC0008316D500831257088316D4008312560851
:101DD0008316D3007A08DA007908D9007808D80089
:101DE0007708D7008A11831253248A157408840057
:101DF0007A08D9007908D8007808D7007708D60083
:101E00008316D501D4014030D3008030D200831234
:101E100051088316D900831250088316D800831204
:101E20004F088316D70083124E088316D6008A11F6
:101E3000831264268A157708F3007808F40079087D
:101E4000F5007A08F6008316A3007908A200780846
:101E5000A1007708A0008A1183123F278A158F30CE
:101E60008316D500FC30D4004130D3007530D20049
:101E70007A08D9007908D8007808D7007708D60002
:101E80008A11831264268A150408F4008310590805
:101E90008316D600831258088316D500831257087C
:101EA0008316D400831256088316D3007A08DA000A
:101EB0007908D9007808D8007708D7008A118312EA
:101EC00053248A15740884007A08D9007908D80048
:101ED0007808D7007708D6008A150A16002F51080F
:101EE0008316D100831250088316D00083124F0846
:101EF0008316CF0083124E088316CE00D501D4017D
:101F0000D3018130D2008A11831297258A15770870
:101F1000E3007808E4007908E5007A08E600831415
:101F200066088316D600831265088316D5008312CF
:101F300064088316D400831263088316D300DA0181
:101F4000D9013430D8008630D7008A118312532447
:101F50008A157708E7007808E8007908E9007A0828
:101F6000EA008316D500831269088316D400831211
:101F700068088316D300831267088316D200DB300B
:101F8000D9000F30D8004930D7008030D6008A11F0
:101F9000831264268A157708EB007808EC0079082C
:101FA000ED007A08EE008316D10083126D088316C7
:101FB000D00083126C088316CF0083126B0883163F
:101FC000CE00D501D4013430D3008630D2008A113E
:101FD000831297258A157A08D1007908D0007808ED
:0C1FE000CF007708CE008A150A16062FE5
:1020000030302E02EC00F0000A30F1000A120E24EB
:102010000A167808ED0030302F026D07E700E8015E
:1020200030303002EC00F0000A30F1000A120E24C9
:102030000A167808ED00303031026D07E9003030C3
:102040003902EC00F0006430F1000A120E240A1686
:102050007808ED0030303A02EF00F0000A30F1006D
:102060000A120E240A1678086D07F00030303B0281
:1020700070078316D301D2000A12831233240A1682
:102080007A08E6007908E5007808E4007708E300BC
:1020900030303C02EC00F0000A30F1000A120E244D
:1020A0000A163D087807D03EF000F1003C30F200FF
:1020B0000A1268270A1678088316D301D2000A127A
:1020C000831233240A16831066088316D6008312FF
:1020D00065088316D500831264088316D400831222
:1020E00063088316D3007A08DA007908D9007808E3
:1020F000D8007708D7000A12831253240A167A08E8
:10210000E6007908E5007808E4007708E3003E0877
:10211000573C031DAE288316D501D4018030D3006F
:102120007F30D200831266088316D90083126508B7
:102130008316D800831264088316D70083126308BD
:102140008316D6000A12831264260A167A08E6005D
:102150007908E5007808E4007708E3008316D501E4
:10216000D401D3018130D200831266088316D900CE
:10217000831265088316D800831264088316D7007B
:10218000831263088316D6000A12831264260A1685
:10219000831055088316D600831254088316D50081
:1021A000831253088316D400831252088316D30077
:1021B0007A08DA007908D9007808D8007708D700BB
:1021C0000A12831253240A167A08D1007908D00023
:1021D0007808CF007708CE005108E6005008E500E7
:1021E0004F08E4004E08E3006808EC006708EB00C5
:1021F000EE013C30ED000A127D2F0A167908FA0034
:1022000078088316D2007908D3000A128312332487
:102210000A16831066088316D60083126508831693
:10222000D500831264088316D400831263088316D2
:10223000D3007A08DA007908D9007808D80077083E
:10224000D7000A12831253240A167708EB00780885
:10225000EC007908ED007A08EE008316D3018312B2
:1022600069088316D2000A12831233240A168310D7
:102270006E088316D60083126D088316D50083126C
:102280006C088316D40083126B088316D3007A0877
:10229000DA007908D9007808D8007708D7000A1240
:1022A000831253240A167A08D1007908D0007808DE
:1022B000CF007708CE0051088316D1008312500852
:1022C0008316D00083124F088316CF0083124E0866
:1022D0008316CE00D501D4013430D3008830D2002B
:1022E0000A128312DC260A16031C7829DC147929C9
:1022F000DC108A150A16032F30303402E800F00093
:102300000A30F1000A120E240A167808E90030306B
:10231000350269078316D301D2000A1283123324CF
:102320000A167A08E6007908E5007808E4007708DC
:10233000E30030303602E800F0000A30F1000A1203
:102340000E240A1637087807D03EEC00F1003C3026
:10235000F2000A1268270A1678088316D301D20001
:102360000A12831233240A16831066088316D600D5
:10237000831265088316D500831264088316D4007F
:10238000831263088316D3007A08DA007908D9002B
:102390007808D8007708D7000A12831253240A1647
:1023A0007A08E6007908E5007808E4007708E30099
:1023B00030303802E800EA016808E9000230EC0039
:1023C0005830EB000A12942F0A167908FA007808A0
:1023D0008316D2007908D3000A12831233240A1616
:1023E000831066088316D600831265088316D5000D
:1023F000831264088316D400831263088316D30003
:102400007A08DA007908D9007808D8007708D70068
:102410000A12831253240A167A08E6007908E500A6
:102420007808E4007708E30066088316D500831275
:1024300065088316D400831264088316D3008312C0
:1024400063088316D200DB30D9000F30D800493042
:10245000D7008030D6000A12831264260A16770845
:10246000E7007808E8007908E9007A08EA008316AE
:10247000D100831269088316D0008312680883167E
:10248000CF00831267088316CE00D501D401343003
:10249000D3008630D2000A12831297250A167A08D2
:1024A000E6007908E5007808E4007708E3006608AC
:1024B000D5006508D4006408D3006308D200510831
:1024C0008316AB00831250088316AA0083124F08AC
:1024D0008316A90083124E088316A8000A128A15D3
:1024E000831255210A168A117A08D1007908D00082
:1024F0007808CF007708CE0066088316AB008312F9
:1025000065088316AA00831264088316A900831243
:1025100063088316A8000A128A15831255210A1629
:102520008A117708E7007808E8007908E9007A0856
:10253000EA0059088316AB00831258088316AA00D4
:10254000831257088316A900831256088316A80021
:102550000A128A15831255210A168A116A088316EF
:10256000D500831269088316D40083126808831685
:10257000D300831267088316D2007A08D90079083D
:10258000D8007808D7007708D6000A12831264268C
:102590000A167708EB007808EC007908ED007A0855
:1025A000EE008316D50083126D088316D4008312C3
:1025B0006C088316D30083126B088316D200831233
:1025C00051088316D900831250088316D80083124D
:1025D0004F088316D70083124E088316D6000A12BE
:1025E000831264260A167A08D1007908D000780888
:1025F000CF007708CE0066088316A3008312650813
:102600008316A200831264088316A1008312630854
:102610008316A0000A1283123F270A167708E700E4
:102620007808E8007908E9007A08EA005908831672
:10263000A300831258088316A2008312570883163A
:10264000A100831256088316A0000A1283123F27A6
:102650000A166A088316D500831269088316D40007
:10266000831268088316D300831267088316D2008A
:102670007A08D9007908D8007808D7007708D600FA
:102680000A12831264260A160408EB00831051080C
:102690008316D600831250088316D50083124F0884
:1026A0008316D40083124E088316D3007A08DA000A
:1026B0007908D9007808D8007708D7000A12831261
:1026C00053240A166B0884007A08D1007908D000D8
:1026D0007808CF007708CE008A150A16092F6A08F5
:1026E000F2006908F1006808F0006708EF000130A7
:1026F000F300741072088316A3007108A20070081A
:10270000A10083126F088316A0007208D10071081F
:10271000D0007008CF0083126F088316CE00D50159
:10272000D401D301D2010A128312DC260A16031C3B
:102730009E2B741480308316A10683128316D10158
:10274000D001CF017E30CE002308D5002208D4006E
:102750002108D3002008D2000A128312DC260A16B0
:10276000031C962C83148316D601D501D4017F3027
:10277000D3002308DA002208D9002108D800200855
:10278000D7000A12831253240A1677088316B00062
:102790007808B1007908B2007A08B3003308D10094
:1027A0003208D0003108CF003008CE00D501D40166
:1027B000D3018030D2000A12831297250A167708B7
:1027C0008316B4007808B5007908B6007A08B70017
:1027D0003708BC003608BB003508BA003408B90019
:1027E0003C08D1003B08D0003A08CF003908CE00A1
:1027F000D501D401D301D2010A128312DC260A16B4
:102800000318042C031D092CF701F801F901FA0142
:102810008A2C83163C08C0003B08BF003A08BE0063
:102820003908BD00BD30C500450884000008C80156
:10283000C7007F304707C9004808CA000318CA0A02
:1028400003104A0CFA00490CF900CB00450884003B
:102850004B0880004008C4003F08C3003E08C20087
:102860003D08C1003C08D1003B08D0003A08CF0029
:102870003908CE004008D5003F08D4003E08D300F8
:102880003D08D2000A12831297250A168310831678
:102890004008D6003F08D5003E08D4003D08D300CC
:1028A0007A08DA007908D9007808D8007708D700C4
:1028B0000A12831253240A167A088316C000790874
:1028C000BF007808BE007708BD004508840080037B
:1028D0004408D1004308D0004208CF004108CE0090
:1028E0004008D5003F08D4003E08D3003D08D20080
:1028F0000A128312DC260A160319802C83162A2C4E
:1029000083164108F7004208F8004308F90044081C
:10291000FA0083127A088316A3007908A2007808C7
:10292000A1007708A0000230F30783128316230862
:10293000D5002208D4002108D3002008D2002308A3
:10294000D9002208D8002108D7002008D6000A1292
:10295000831264260A167A088316AF007908AE003F
:102960007808AD007708AC003730D500BF30D40010
:102970007D30D300D2002F08D9002E08D8002D08B2
:10298000D7002C08D6000A12831264260A1677088C
:102990008316B0007808B1007908B2007A08B30055
:1029A00083103308D6003208D5003108D40030082F
:1029B000D3003D30DA00AA30D9009330D8008130FE
:1029C000D7000A12831253240A167A088316A70026
:1029D0007908A6007808A5007708A4002708D50084
:1029E0002608D4002508D3002408D2002F08D900D7
:1029F0002E08D8002D08D7002C08D6000A12831202
:102A000064260A1677088316B0007808B1007908A2
:102A1000B2007A08B30083103308D6003208D5001C
:102A20003108D4003008D300EE30DA005030D9003D
:102A30003330D8008130D7000A12831253240A168B
:102A40007A088316A7007908A6007808A5007708F9
:102A5000A400D501D401D3017F30D2002F08D900C2
:102A60002E08D8002D08D7002C08D6000A12831291
:102A700064260A1677088316B0007808B100790832
:102A8000B2007A08B30083103308D6003208D500AC
:102A90003108D4003008D3000A30DA008D30D90074
:102AA000B130D8008130D7000A12831253240A169D
:102AB0007A088316AB007908AA007808A90077087D
:102AC000A8002B08D5002A08D4002908D30028081C
:102AD000D2002F08D9002E08D8002D08D7002C08C6
:102AE000D6000A12831264260A1677088316B000ED
:102AF0007808B1007908B2007A08B300831033086F
:102B0000D6003208D5003108D4003008D300EE30AA
:102B1000DA005030D9003330D8008130D7000A12A3
:102B2000831253240A167A088316AB007908AA0088
:102B30007808A9007708A8002308D5002208D40047
:102B40002108D3002008D2002708D9002608D80081
:102B50002508D7002408D6000A12831264260A1614
:102B600077088316B0007808B1007908B2007A08B7
:102B7000B300D1003208D0003108CF003008CE00B9
:102B80002B08D5002A08D4002908D3002808D20031
:102B90000A12831297250A167A088316A700790865
:102BA000A6007808A5007708A400F31C072ED5011D
:102BB000D401D3018030D2002708D9002608D800DC
:102BC0002508D7002408D6000A12831264260A16A4
:102BD0008314DB308316D6000F30D5004930D40083
:102BE0007F30D3007A08DA007908D9007808D80055
:102BF0007708D7000A12831253240A167A0883161C
:102C0000A7007908A6007808A5007708A400741C1E
:102C10000B2E8030A506731C2B2E8314DB30D600C0
:102C20000F30D5004930D4007F30D3002708DA00B8
:102C30002608D9002508D8002408D7000A128312D4
:102C400053240A167A088316A7007908A600780884
:102C5000A5007708A4002408F7002508F800260836
:102C6000F9002708FA007A088312EE007908ED00CF
:102C70007808EC007708EB006B08F7006C08F800A8
:102C80006D08F9006E08FA0000345108EA00500897
:102C9000E9004F08E8004E08E7006F237A08D100EA
:102CA0007908D0007808CF007708CE008314DB3095
:102CB0008316D6000F30D5004930D4007F30D300C2
:102CC000831251088316DA00831250088316D90044
:102CD00083124F088316D80083124E088316D7003C
:102CE0000A12831253240A167708E7007808E800CE
:102CF0007908E9007A08EA008316D100831279087E
:102D00008316D000831278088316CF0083127708C9
:102D10008316CE00DB30D5000F30D4004930D3000D
:102D20008030D2000A12831297250A167708EB002A
:102D30007808EC007908ED007A08EE008316D500DB
:102D4000831279088316D400831278088316D3007F
:102D5000831277088316D200D901D8013430D70006
:102D60008630D6000A12831264260A167708EF000E
:102D70007808F0007908F1007A08F20083107A08E8
:102D80008316D6007908D5007808D4008312770816
:102D90008316D300DA01D901D8017E30D7000A1298
:102DA000831253240A167A088316D1007908D000BA
:102DB0007808CF007708CE000A1283121D270A1662
:102DC0007808CD008A150A160C2FEB010A12C121D2
:102DD0000A163F08F3000A12B9210A164008F30048
:102DE0000A12B9210A162F30F3000A12B9210A1665
:102DF0004108F3000A12B9210A164208F3000A1228
:102E0000B9210A16303031020139013C031D1B2F54
:102E1000E30163080A1274200A1600380319162FFA
:102E2000E30AF3000A12B9210A16092F83160612C3
:102E3000831206162D2FE30163080A127C200A165E
:102E400000380319292FE30AF3000A12B9210A16E0
:102E50001C2F83160612831206122E08F3000A1284
:102E6000B9210A162F08F3000A12B9210A163A30BE
:102E7000F3000A12B9210A163008F3000A12B92128
:102E80000A163108F3000A12B9210A163A30F30083
:102E90000A12B9210A163208F3000A12B9210A16D9
:102EA0003308F3000A12B9210A162030F3000A127F
:102EB000B9210A168A150A16102F6910E801E801CF
:102EC0006808E80A003A0319742F63306807EA00BB
:102ED0000A123F230A166A088400780880006808EE
:102EE000033C031C0030602F6918992F0A123F23FE
:102EF0000A167808E7006308473C031D8F2F640813
:102F0000503C031D8F2F6508473C031D8F2F66081B
:102F1000473C031D8F2F6708413C03196914E80AD9
:102F20006408E3006508E4006608E5006708E60059
:102F3000742F003069180130F8008A150A161A2F0C
:1030000055088316A300831254088316A200831266
:1030100053088316A100831252088316A0000A12D7
:103020008A1183123F270A168A157708E700780865
:10303000E8007908E9007A08EA0051088316AB0035
:10304000831250088316AA0083124F088316A90022
:1030500083124E088316A8000A12831255210A16FD
:103060006A088316D500831269088316D400831278
:1030700068088316D300831267088316D2007A0883
:10308000D9007908D8007808D7007708D6000A1246
:103090008A11831264260A168A157708EB007808CD
:1030A000EC007908ED007A08EE0059088316A300B9
:1030B000831258088316A200831257088316A100B2
:1030C000831256088316A0000A128A1183123F2722
:1030D0000A168A150408EF0083146E088316D600BA
:1030E00083126D088316D50083126C088316D400F2
:1030F00083126B088316D3007A08DA007908D900A6
:103100007808D8007708D7000A128A11831253244E
:103110000A168A156F0884007A08D9007908D80041
:103120007808D7007708D60051088316A3008312C9
:1031300050088316A20083124F088316A100831241
:103140004E088316A0000A128A1183123F270A161E
:103150008A1559088316D100831258088316D000A7
:10316000831257088316CF00831256088316CE00A9
:103170007A08D5007908D4007808D3007708D200FF
:103180000A128A11831297250A168A157A08D10025
:103190007908D0007808CF007708CE00550883164C
:1031A000AB00831254088316AA00831253088316B7
:1031B000A900831252088316A8000A12831255210F
:1031C0000A1651088316D100831250088316D000C6
:1031D00083124F088316CF0083124E088316CE0049
:1031E0007A08D5007908D4007808D3007708D2008F
:1031F0000A128A11831297250A168A157A08D100B5
:103200007908D0007808CF007708CE005108EA008E
:103210005008E9004F08E8004E08E7008A116F23C4
:103220008A157708E7007808E8007908E9007A0845
:10323000EA008316D100831269088316D000831236
:1032400068088316CF00831267088316CE00DB3030
:10325000D5000F30D4004930D3008030D2000A129C
:103260008A11831297250A168A157708EB007808C9
:10327000EC007908ED007A08EE008316D500831281
:103280006D088316D40083126C088316D300831252
:103290006B088316D200D901D8013430D7008630AC
:1032A000D6000A128A11831264260A168A157A0831
:1032B000D1007908D0007808CF007708CE00DC1C58
:1032C00063298030CF0683108316D601D5013430B0
:1032D000D4008630D300831251088316DA0083129B
:1032E00050088316D90083124F088316D800831222
:1032F0004E088316D7000A128A11831253240A1625
:103300008A157708E7007808E8007908E9007A0864
:10331000EA0083106A088316D600831269088316B0
:10332000D500831268088316D400831267088316B9
:10333000D300DA01D901D8017E30D7000A128A11F0
:10334000831253240A168A157A088316D100790845
:10335000D0007808CF007708CE000A128A118312B5
:103360001D270A168A157908CC007808CB008A1523
:103370000A160E2F3E08453C031DEB29303039025A
:10338000EA006430F0006A08F1000A128A110E2483
:103390000A168A157808EB0030303A02EC000A3041
:1033A000F0006C08F1000A128A110E240A168A1520
:1033B00078086B07ED0030303B026D07EF00F1003D
:1033C0001430F2000A128A1168270A168A15780842
:1033D0004A3EE400172A30303902EA006430F00037
:1033E0006A08F1000A128A110E240A168A15780852
:1033F000EB0030303A02EC000A30F0006C08F100CB
:103400000A128A110E240A168A1578086B07ED0035
:1034100030303B026D07EF00F1001430F2000A1269
:103420008A1168270A168A157808493CE40030306A
:103430003402EA000A30F0006A08F1000A128A1128
:103440000E240A168A157808EB00303035026B0717
:10345000ED00F1000A30F2000A128A1168270A16FC
:103460008A1578084A3EE5003E08453C031D672A58
:1034700030303902EA006430F0006A08F1000A12C4
:103480008A110E240A168A157808EB0030303A02A9
:10349000EC000A30F0006C08F1000A128A110E24C8
:1034A0000A168A1578086B07ED0030303B026D076D
:1034B000EF00F1001430F2000A128A1168270A1690
:1034C0008A150310F70C7708303EE600952A303055
:1034D0003902EA006430F0006A08F1000A128A1129
:1034E0000E240A168A157808EB0030303A02EC00F8
:1034F0000A30F0006C08F1000A128A110E240A1634
:103500008A1578086B07ED0030303B026D07EF003D
:10351000F1001430F2000A128A1168270A168A157F
:103520000310F70C7708393CE6003508E7003E0841
:10353000453C031DDC2A30303B020139003A031DB3
:10354000BE2A30303C02EA000A30F0006A08F1007E
:103550000A128A110E240A168A157808EB003030F8
:103560003D026B07ED00F1000530F2000A128A11EE
:1035700068270A168A157808E300DB2A30303C02F7
:10358000EA000A30F0006A08F1000A128A110E24DB
:103590000A168A157808EB0030303D026B073C3E76
:1035A000ED00F1000530F2000A128A1168270A16B0
:1035B0008A157808E3001D2B30303B020139013CAD
:1035C000031D002B30303C02EA000A30F0006A088C
:1035D000F1000A128A110E240A168A157808EB00E7
:1035E00030303D026B07ED00F1000530F2000A12A9
:1035F0008A1168270A168A1578080B3CE3001D2BF0
:1036000030303C02EA000A30F0006A08F1000A1289
:103610008A110E240A168A157808EB0030303D0214
:103620006B07ED00F1000530F2000A128A116827DD
:103630000A168A157808173CE30041306307E80052
:1036400030303602EA000A30F0006A08F1000A124F
:103650008A110E240A168A157808EB0030303702DA
:103660006B07ED00F1000530F2000A128A1168279D
:103670000A168A157808E9000310690D413EE90031
:1036800030303602EA000A30F0006A08F1000A120F
:103690008A110E240A168A157808EB00303037029A
:1036A0006B07ED00F1000530F2000A128A1168275D
:1036B0000A168A157708E3006308023C031CE90A2E
:1036C0006308023C031D692B30303802053C031CA3
:1036D000E90A6408B4006508B5006608B600670822
:1036E000B7006808BC006908BD008A150A16122FC9
:1036F000E3010A128A113F230A168A156308043C63
:10370000031C892B0A128A118C230A168A15E30AD4
:103710007E2B0A128A113F230A168A15303078024E
:10372000C7000A128A113F230A168A150A128A1143
:103730003F230A168A157808C8000A128A113F2307
:103740000A168A157808C900C7080319302C0A120E
:103750008A113F230A168A157808C3000A128A11B3
:103760003F230A168A157808C5000A128A113F23DA
:103770000A168A157808C60046082E3C031DC42B7D
:103780004508C6003030C5004508303C031DD22B2B
:103790004608393C031DD12B3030C6003130C500FE
:1037A000D22BC60A30304502E4000A30F00064082B
:1037B000F1000A128A110E240A168A157808E5000B
:1037C000303046026507CA000A128A118C230A1695
:1037D0008A150A128A113F230A168A157808C3002F
:1037E0000A128A113F230A168A157808C4000A12A1
:1037F0008A113F230A168A157808C5000A128A1111
:103800003F230A168A157808C60043082E3C031D7C
:103810000F2C3030C6002030C500C400C30044085F
:103820002E3C031D192C4308C6002030C500C400DF
:10383000C30045082E3C031D242C4408C600430841
:10384000C5002030C400C30046082E3C031D302CA8
:103850004508C6004408C5004308C4002030C30022
:103860008A150A16422F20306C1E3030ED006B088E
:10387000F700EB1F422CF709F70A7708EB002D3011
:10388000ED00EC176B08F1006430F2000A128A11A7
:1038900068270A168A157708EB0030307807EE00A3
:1038A0006B08F1000A30F2000A128A1168270A1622
:1038B0008A1530307707F00030307807EF006D0858
:1038C000F700EC1D652CEC1F6C116C1A722CEC1FB0
:1038D0008D2C6C198D2C7708EE00EC188D2C770848
:1038E000EF008D2C30306E02031D8D2C7708EE001A
:1038F0002030ED00EC1D802C6C11EC14EC1FEC1052
:1039000030306F02031D8D2C7708EF002030EE0061
:10391000EC1D802CEC10EC1F6C106C1D962C6D08AF
:10392000F3000A128A11B9210A168A15EC1C9F2C81
:103930006E08F3000A128A11B9210A168A156C1C46
:10394000A82C6F08F3000A128A11B9210A168A15E9
:103950007008F3000A128A11B9210A168A15003478
:103960000408F200EC1FBC2CF217721EF20AEB09DD
:10397000EC09EB0A0319EC0A6C0EF038EE00EE07C6
:10398000E23EEF00323EF1006C080F39EF07EF071F
:10399000F107E93EF000F007F0076B0E0F39F00772
:1039A000F107F00DF10DF109F10D6B080F39F10779
:1039B000EE0D0730ED000A30F107F003031CDC2C9C
:1039C000F007EF03031CE02CEF07EE03031CE42CCD
:1039D000EE07ED03031CE82C6D3084000730720500
:1039E000721384037205031DFC2C721A840A721A66
:1039F000FC2C2030F700192D8407713004020319C4
:103A000072170008F700031D0D2D721B0D2D721A81
:103A1000252DF2190D2D2030182DF21F152D2D30CA
:103A2000F70084037213F213192DF215721230305D
:103A3000F707EC010408EB007708F3000A128A117B
:103A4000B9210A168A156B088400840A721FFD2C9E
:103A50008A150A16F02D4030EB000A128A11C12196
:103A60000A168A153408F3000A128A11B9210A16B7
:103A70008A153508F3000A128A11B9210A168A1527
:103A80003608F3000A128A11B9210A168A15370876
:103A9000F3000A128A11B9210A168A153C08F300AC
:103AA0000A128A11B9210A168A153D08F3000A1272
:103AB0008A11B9210A168A154930EB000A128A11B7
:103AC000C1210A168A156A08F63E0318FD2D0A3E22
:103AD000002E5C1CA32DC7080319A32DEB016B0856
:103AE0000A128A1184200A168A1500380319802DBB
:103AF000EB0AF3000A128A11B9210A168A156F2DF2
:103B00004308F3000A128A11B9210A168A154408DB
:103B1000F3000A128A11B9210A168A154508F30022
:103B20000A128A11B9210A168A154608F3000A12E8
:103B30008A11B9210A168A156D30F3000A128A110A
:103B4000B9210A168A15FD2D5C1CC92DC708031959
:103B5000C92D4808F3000A128A11B9210A168A15DC
:103B60004908F3000A128A11B9210A168A15EB01D5
:103B70006B080A128A118B200A168A15003803195D
:103B8000C92DEB0AF3000A128A11B9210A168A1507
:103B9000B82DFD2D5C1CE62DC7080319E62DEB01A1
:103BA0006B080A128A1195200A168A150038031923
:103BB000E12DEB0AF3000A128A11B9210A168A15BF
:103BC000D02D4A08EB001130EC003324FD2D5C1C95
:103BD000FC2D033084004C08EC004B08EB00B02CAB
:103BE0002F30F3000A128A11B9210A168A154D08DE
:103BF000EB001330EC003324FD2D8A150A16A02F9C
:103C00000A108A140A158207692D692D692DA42DC1
:103C1000A42DCA2DCA2DE72DE72DE72D84011F30D5
:103C2000830583161F149F141F159F1107309C00D6
:103C30001C0883120D130C30831699002230980053
:103C4000903083129800AC01AD01C701CB01CC01CB
:103C5000CD01DC10FF30DD00E00162140A128A1190
:103C6000CB290A168A152D082C020319A12FE00171
:103C7000621CB32E0A128A119C210A168A15E301CE
:103C800063080A128A119F200A168A150038031940
:103C9000512EE30AF3000A128A11B9210A168A1575
:103CA000402E0A128A114F230A168A15F8080319A2
:103CB0005B2E00305C2E0130F8007818612E621007
:103CC000622E6214621C892E4030EB000A128A11A7
:103CD000C1210A168A15E30163080A128A11AD2070
:103CE0000A168A15003803197D2EE30AF3000A121A
:103CF0008A11B9210A168A156C2E0430E300FA30B5
:103D0000E4000A128A1112210A168A15E30B7F2E8B
:103D1000B22E4030EB000A128A11C1210A168A1510
:103D2000E30163080A128A11BB200A168A150038BB
:103D30000319A22EE30AF3000A128A11B9210A1606
:103D40008A15912E0430E300FA30E4000A128A1139
:103D500012210A168A15E30BA42E0A128A119C213D
:103D60000A168A15A02F0A128A114F230A168A15DD
:103D7000F808031DDE2EEB010A128A11C1210A1672
:103D80008A15E30163080A128A11C9200A168A15E6
:103D900000380319D32EE30AF3000A128A11B9215D
:103DA0000A168A15C22E0430E300FA30E4000A1223
:103DB0008A1112210A168A15E30BD52E0A128A11CE
:103DC000982B0A168A1530303002E400F0000A30D1
:103DD000F1000A128A110E240A168A1530303102B7
:103DE0007807E1005A08610203190E2F6108DA0012
:103DF0000A1200280A160A12302B0A160A12F62C8A
:103E00000A168A1100288A150A126F2F0A168A11BB
:103E10007C298A158A11452E8A1500288A11E52EDB
:103E20008A15BA295B0832020319442F5C1C442FFF
:103E30008A115D2F8A15F808031D412FEB010A1224
:103E40008A11C1210A168A15E30163080A128A1130
:103E5000D6200A168A1500380319362FE30AF30014
:103E60000A128A11B9210A168A15252F0430E30097
:103E7000FA30E4000A128A1112210A168A15E30B9D
:103E8000382F782B3208DB004730EB000A128A11FA
:103E9000C1210A168A15C7080319642F5C1C642FF8
:103EA0004A08013C031C642F2130F3000A128A11D6
:103EB000B9210A168A158316061183120615831670
:103EC0008611831286117F2F5C1D6E2F3F30F30009
:103ED0000A128A11B9210A168A15752F2030F300AB
:103EE0000A128A11B9210A168A158316061183123D
:103EF000061183168611831286150430DC063030D5
:103F00003202E400F0000A30F1000A128A110E2495
:103F10000A168A157808E500303033027807F70072
:103F20000310F70C7708E800F1000A30F2000A12DB
:103F30008A1168270A168A157708E900EA002B2DEE
:103F4000D42F6008313C0318BD2F0A128A119C211E
:103F50000A168A15E30163080A128A11E3200A1679
:103F60008A1500380319BC2FE30AF3000A128A11DC
:103F7000B9210A168A15AB2FBE2FE00A83168612C6
:103F8000831286163230E4000A128A1112210A16B0
:103F90008A1583168612831286123230E4000A12C2
:0C3FA0008A1112210A168A15332E6300C4
:02400E00723FFF
:00000001FF
